:1000000012C0189518951895189518951895189563
:1000100025C66BC2189518951895189518951895BA
:100020001895189518958FE58DBFC8E3E0E24E2E20
:1000300084E08EBFD4E0F4E05F2EA89584B7082E4C
:10004000877F84BF88E1992781BD91BDEEEFF3E002
:10005000A0E6B0E088278D933197E9F76624A09851
:10006000A89AA198A99AA298AA9A8FEF81BB8FEF1C
:1000700087BB86E886B980E487B981E08093620017
:1000800000916200063010F009F015C08BE090E09E
:10009000A2E6B0E0AD90BB24A3E6B0E0AA0CBB1C86
:1000A000AA0DBB1D8D939C93A2E6B0E08C918F5F4F
:1000B0008C9308F4E5CFEAE1F0E0A2E9B0E091E04A
:1000C000B6DA989957C081E080936200009162008F
:1000D000083C10F009F04EC000916200063909F0AA
:1000E0003CC080918C00806880938C00A2E9B0E0D5
:1000F0008C9198E089278C93EAE1F0E0A2E9B0E0E6
:1001000091E07BE783DA00919200003009F00EC0A5
:1001100092989698C798C2989098C6989798C598BC
:10012000939A949A919A959AC09AC19A0091920042
:10013000083009F00EC0929A969AC79AC29A909A7D
:10014000C69A979AC59A9398949891989598C098BA
:10015000C1988CED95E01CDA0DC0989B01C00AC0D7
:100160008AE090E015DAA2E6B0E08C918F5F8C9384
:1001700008F4ACCFE4E1F0E0A0E1B0E055DA0F3FE5
:1001800009F05AC08EE190E0A5E7B0E08D939C9312
:1001900084E190E0A3E7B0E08D939C938CE390E042
:1001A000ABE7B0E08D939C9382E390E0A9E7B0E0E9
:1001B0008D939C9380E0809392008BEB80938F00D3
:1001C0008BEB80939000E0E0F0E0A3E7B0E092E0FA
:1001D0007BE71CDAE5E0F0E0A5E7B0E092E07BE742
:1001E00015DAEAE0F0E0A9E7B0E092E07BE70EDAAA
:1001F000EEE0F0E0ABE7B0E092E07BE707DAE0E1C9
:10020000F0E0AFE8B0E091E07BE700DAE1E1F0E0B8
:10021000A0E9B0E091E07BE7F9D9EAE1F0E0A2E9FA
:10022000B0E091E07BE7F2D9E4E1F0E0A0E1BB27A8
:1002300084E68C937BE7E7D9E0E0F0E0A3E7B0E069
:1002400092E0F5D9E5E0F0E0A5E7B0E092E0EFD983
:10025000EAE0F0E0A9E7B0E092E0E9D9EEE0F0E012
:10026000ABE7B0E092E0E3D9E0E1F0E0AFE8B0E086
:1002700091E0DDD9E1E1F0E0A0E9B0E091E0D7D98B
:1002800082E083BF80E08FBD81E08EBD789489B726
:10029000816089BF89B7846089BF82E083BF81E0C4
:1002A0008EBD379A00916200083210F009F001C04B
:1002B00073C0882783BF8EB5887F8EBD07B1007F4E
:1002C000056007B974D9A1E7B0E08D939C93A1E7CD
:1002D000B0E00D911C910A3C53E0150714F009F0B1
:1002E00001C005C080918C00806180938C000FEF6D
:1002F00013E0A1E7B0E04D915C91041B150BA1E761
:10030000B0E00D931C93A1E7B0E00D911C914AE081
:1003100050E0FBD8A1E7B0E04D935C93A1E7B0E0DB
:100320000D911C91043650E0150714F009F001C03E
:1003300006C084E690E0A1E7B0E08D939C9307B1FE
:10034000007F046007B933D9A7E7B0E08D939C9391
:10035000A7E7B0E00D911C91083E53E0150714F09B
:1003600009F001C005C080918C00886080938C00EA
:10037000A7E7B0E00D911C91073E53E0150714F07C
:1003800009F001C006C087EE93E0A7E7B0E08D93C7
:100390009C9380E08093620082E083BF81E08EBD09
:1003A000A5E7B0E04D915C91A3E7B0E00D911C9101
:1003B0000417150708F021C0A3E7B0E04D915C9148
:1003C000A1E7B0E00D911C910417150714F009F096
:1003D00003C081E080937D00A5E7B0E04D915C9182
:1003E000A1E7B0E00D911C91041715070CF001C0B6
:1003F00003C080E080937D0020C0A3E7B0E04D9172
:100400005C91A1E7B0E00D911C91041715070CF069
:1004100001C003C081E080937D00A5E7B0E04D916D
:100420005C91A1E7B0E00D911C910417150714F041
:1004300009F003C080E080937D0000917D000130D1
:1004400081E009F080E08F93ACE8B0E08C9184FB10
:1004500081E00EF080E09F91892B882309F402C08F
:10046000C39A01C0C398ABE7B0E04D915C91A9E796
:10047000B0E00D911C910417150708F011C0A9E711
:10048000B0E04D915C91A7E7B0E00D911C9104178D
:10049000150714F009F003C081E080937E0010C0BE
:1004A000A9E7B0E04D915C91A7E7B0E00D911C91F8
:1004B000041715070CF001C003C081E080937E0093
:1004C00000917E00013081E009F080E08F93ACE87C
:1004D000B0E08C9183FB81E00EF080E09F91892B4E
:1004E000882309F401C0C49ADDCE0F921F922F9287
:1004F0003F924F925F927F92AF92BF920F931F9362
:100500002F933F934F935F936F937F938F939F931B
:10051000AF93BF93CF93DF93EF93FF938FB78F93F7
:1005200000918B00003081E009F480E08F93ACE80B
:10053000B0E08C9185FB81E00EF480E09F918923EF
:10054000882309F403C0ADE8B0E0CED7ADE8B0E051
:100550000D911C9108355BE1150710F009F001C001
:1005600009C080E090E0ADE8B0E08D939C9380E01E
:1005700080938B00882783BF00918B00003009F0A7
:1005800011C0A1E7B0E08D919C91A5E8B0E08D93FA
:100590009C93A7E7B0E08D919C91A7E8B0E08D9384
:1005A0009C934FC0013009F011C0A3E7B0E08D91DA
:1005B0009C91A5E8B0E08D939C93A7E7B0E08D9166
:1005C0009C91A7E8B0E08D939C933BC0023009F06A
:1005D00011C0A5E7B0E08D919C91A5E8B0E08D93A6
:1005E0009C93A7E7B0E08D919C91A7E8B0E08D9334
:1005F0009C9327C0033009F011C0A1E7B0E08D91B2
:100600009C91A5E8B0E08D939C93A9E7B0E08D9113
:100610009C91A7E8B0E08D939C9313C0043009F03F
:1006200010C0A1E7B0E08D919C91A5E8B0E08D935A
:100630009C93ABE7B0E08D919C91A7E8B0E08D93DF
:100640009C93ACE8B0E08C9181FB0EF44FC0A5E820
:10065000B0E08D919C91AFE7B0E08D939C93AFE7B4
:10066000B0E08D919C91A3E8B0E08D939C9383E0E2
:10067000809363004091630001E0041710F009F0DB
:1006800025C0AFE7B0E00D911C914AE050E03DD7A6
:10069000A3E6B0E0AD90BB24A3E6B0E0AA0CBB1C7F
:1006A000AA0DBB1D0D931C93AFE7B0E00D911C91FB
:1006B0004AE050E02AD7AFE7B0E04D935C938091D9
:1006C000630081508093630008F0D4CFA3E8B0E0CA
:1006D0000D911C91043650E015070CF401C006C0C2
:1006E0008BE090E0A5E6B0E08D939C93ACE8B0E0A1
:1006F0008C9180FB0EF44FC0A7E8B0E08D919C91E7
:10070000A1E8B0E08D939C93A1E8B0E08D919C911D
:10071000A3E8B0E08D939C9386E0809363004091C2
:10072000630004E0041710F009F025C0A1E8B0E070
:100730000D911C914AE050E0E8D6A3E6B0E0AD9000
:10074000BB24A3E6B0E0AA0CBB1CAA0DBB1D0D93F5
:100750001C93A1E8B0E00D911C914AE050E0D5D681
:10076000A1E8B0E04D935C93809163008150809349
:10077000630008F0D4CFA3E8B0E00D911C910436DB
:1007800050E015070CF401C006C08BE090E0ABE62A
:10079000B0E08D939C9300919200003009F007C067
:1007A0009398949891989598C098C19806C0939AF8
:1007B000949A919A959AC09AC19AA0E6B0E08C91C9
:1007C0008F5F8C9300916000063010F009F001C03B
:1007D00003C081E08093600080E08093610090D14D
:1007E000A4E6B0E08C9180FBA2E3B0E08C9182F9AA
:1007F0008C9386D1A4E6B0E08C9180FBA2E3B0E0BC
:100800008C9186F98C937CD1A4E6B0E08C9180FB2E
:10081000A8E3B0E08C9187F98C9372D1A4E6B0E0A4
:100820008C9180FBA8E3B0E08C9182F98C9368D125
:10083000A4E6B0E08C9180FBA2E3B0E08C9180F95B
:100840008C935ED1A4E6B0E08C9180FBA8E3B0E08D
:100850008C9186F98C9354D1A4E6B0E08C9180FB06
:10086000A2E3B0E08C9187F98C9300916000013095
:1008700009F02FC000919200003009F013C0919A46
:10088000ACE8B0E08C9181FB0EF40AC0AFE8B0E0B8
:100890008C9183FBA8E3B0E08C9185F98C9301C027
:1008A000C59A16C09198ACE8B0E08C9181FB0EF42B
:1008B0000EC0AFE8B0E08C9183FBA8E3B0E08C9170
:1008C00085F98C9388B390E2892788BB01C0C598CD
:1008D000F9C0023009F02FC000919200003009F0F9
:1008E00013C0949AACE8B0E08C9181FB0EF40AC07E
:1008F000AFE8B0E08C9182FBA8E3B0E08C9185F981
:100900008C9301C0C59A16C09498ACE8B0E08C9165
:1009100081FB0EF40EC0AFE8B0E08C9182FBA8E33F
:10092000B0E08C9185F98C9388B390E2892788BBDD
:1009300001C0C598C7C0033009F02FC000919200D4
:10094000003009F013C0939AACE8B0E08C9181FBC1
:100950000EF40AC0AFE8B0E08C9181FBA8E3B0E0F0
:100960008C9185F98C9301C0C59A16C09398ACE818
:10097000B0E08C9181FB0EF40EC0AFE8B0E08C913A
:1009800081FBA8E3B0E08C9185F98C9388B390E269
:10099000892788BB01C0C59895C0043009F02FC0D5
:1009A00000919200003009F013C0C19AACE8B0E0A9
:1009B0008C9180FB0EF40AC0A0E9B0E08C9183FB1F
:1009C000A8E3B0E08C9185F98C9301C0C59A16C05C
:1009D000C198ACE8B0E08C9181FB0EF40EC0A0E9A8
:1009E000B0E08C9183FBA8E3B0E08C9185F98C9307
:1009F00088B390E2892788BB01C0C59863C00530E1
:100A000009F02FC000919200003009F013C0C09A85
:100A1000ACE8B0E08C9180FB0EF40AC0A0E9B0E035
:100A20008C9182FBA8E3B0E08C9185F98C9301C096
:100A3000C59A16C0C098ACE8B0E08C9181FB0EF46A
:100A40000EC0A0E9B0E08C9182FBA8E3B0E08C91ED
:100A500085F98C9388B390E2892788BB01C0C5983B
:100A600031C0063009F02EC000919200003009F02C
:100A700013C0959AACE8B0E08C9180FB0EF40AC0EC
:100A8000A0E9B0E08C9181FBA8E3B0E08C9185F9FE
:100A90008C9301C0C59A16C09598ACE8B0E08C91D3
:100AA00081FB0EF40EC0A0E9B0E08C9181FBA8E3BD
:100AB000B0E08C9185F98C9388B390E2892788BB4C
:100AC00001C0C59882E083BF8F918FBFFF91EF91E6
:100AD000DF91CF91BF91AF919F918F917F916F9156
:100AE0005F914F913F912F911F910F91BF90AF90C8
:100AF0007F905F904F903F902F901F900F90189590
:100B0000A0E6B0E0AD90BB24A3E6B0E0AA0CBB1C0D
:100B1000AA0DBB1D0C9147E0049FA4E6B0E00C9227
:100B20000091610040916400040FA4E6B0E00C93D2
:100B300000919200003009F00AC0ECE6FBE0A4E668
:100B4000B0E08C919927A4E6B0E054D509C0E4EE5A
:100B5000FBE0A4E6B0E08C919927A4E6B0E04AD58A
:100B6000A1E6B0E08C918F5F8C93089500000000A7
:100B7000000001010000010101010000010000016D
:100B80000000000000010100010000010100000060
:100B90000100000100000001000000000000000052
:100BA0000101010100000000000000000000000140
:100BB0000000010101010101000101010101010128
:100BC000010101000000010101000100010000011C
:100BD000010100000000010100000000010101010D
:100BE00000010000010101010101000001010000FC
:100BF00000000101000101000101010101000001EB
:100C000000010100000101010001010001010100DA
:100C100001010101010101010000000001010101C8
:100C200001010101010101000101000000000000BB
:100C300001000000000000000000000101010000B0
:100C4000000100010001010000000101010100009C
:100C50000101010100000000010001000F921F923C
:100C60002F923F924F925F927F92AF92BF920F93DB
:100C70001F932F933F934F935F936F937F938F9324
:100C80009F93AF93BF93CF93DF93EF93FF938FB770
:100C90008F93A2E6B0E08C918F5F8C938EB5887FA6
:100CA0008EBDA3E3B0E00C9100FB81E00EF480E088
:100CB0008F93ACE8B0E08C9187FB81E00EF480E08C
:100CC0009F9189238F93A3E3B0E00C9101FB81E016
:100CD0000EF080E09F9189238F93A3E3B0E00C9105
:100CE00002FB81E00EF080E09F918923882309F4C4
:100CF00001C0E3D0ACE8B0E08C9182FB81E00EF063
:100D000080E08F93A3E3B0E00C9100FB81E00EF054
:100D100080E09F918923882309F406C0999901C036
:100D20000DD39A9901C05BD3A3E3B0E00C9100FB13
:100D300081E00EF480E08F93A3E3B0E00C9101FB1F
:100D400081E00EF480E09F9189238F9300918B00C6
:100D5000003081E009F080E09F9189238F93ACE817
:100D6000B0E08C9186FB81E00EF480E09F918923B6
:100D7000882309F401C08CD3A3E3B0E00C9100FBFD
:100D800081E00EF480E08F93A3E3B0E00C9102FBCE
:100D900081E00EF480E09F9189238F9300918B0076
:100DA000003081E009F080E09F9189238F93ACE8C7
:100DB000B0E08C9186FB81E00EF480E09F91892366
:100DC000882309F401C07AD3A3E3B0E00C9100FBBF
:100DD00081E00EF080E08F93A3E3B0E00C9101FB83
:100DE00081E00EF080E09F9189238F93A3E3B0E030
:100DF0000C9102FB81E00EF080E09F918923882313
:100E000009F405C080918C008F7780938C00989BAB
:100E100005C080918C008F7B80938C00A3E3B0E0B1
:100E20000C9101FB81E00EF480E08F93A3E3B0E02E
:100E30000C9102FB81E00EF480E09F91892B8F934F
:100E400000918B00003081E009F080E09F918923C0
:100E5000882309F412C080E080937D0080E08093B5
:100E60007E00C398C49880918C008F7E80938C0004
:100E700080918C00877F80938C0081E08EBD82E022
:100E800083BF8F918FBFFF91EF91DF91CF91BF9182
:100E9000AF919F918F917F916F915F914F913F9112
:100EA0002F911F910F91BF90AF907F905F904F90C7
:100EB0003F902F901F900F901895789489B781607C
:100EC00089BF82E083BF80918C00846080938C0016
:100ED00080918C00806880938C0080E090E0ADE889
:100EE000B0E08D939C93A5E7B0E04D915C91A3E7B2
:100EF000B0E00D911C910417150781E009F080E026
:100F00008F93ABE7B0E04D915C91A9E7B0E00D9114
:100F10001C910417150781E009F080E09F91892B4F
:100F2000882309F401C0FDD0ABE8B0E08C918F5F5D
:100F30008C9300918B00043010F009F001C003C0C5
:100F400080E080938B0000918B00003009F043C05B
:100F500080918C00826080938C0080918C008160F5
:100F600080938C008AE090E0A5E6B0E08D939C939E
:100F70008AE090E0A7E6B0E08D939C938AE090E051
:100F8000A9E6B0E08D939C938AE090E0ABE6B0E0F8
:100F90008D939C938AE090E0ADE6B0E08D939C93B6
:100FA0008AE090E0AFE6B0E08D939C9380918C0056
:100FB0008B7F80938C0084EF91E0EAD28EB5887F9E
:100FC0008EBD882783BFEEE0F0E0ABE7B0E092E0B3
:100FD0007BE71CD39BC0013009F01BC080918C00C3
:100FE000826080938C0081E090E0A9E6B0E08D9370
:100FF0009C938DE090E0A7E6B0E08D939C9380E019
:1010000090E0A5E6B0E08D939C9384EF91E0C0D290
:101010007DC0023009F027C080918C0082608093EF
:101020008C0081E090E0A9E6B0E08D939C938EE087
:1010300090E0A7E6B0E08D939C9380E090E0A5E679
:10104000B0E08D939C9384EF91E0A2D28EB5887F1F
:101050008EBD882783BFE0E0F0E0A3E7B0E092E038
:101060007BE7D4D253C0033009F027C080918C00B5
:10107000816080938C0082E090E0AFE6B0E08D93D9
:101080009C938DE090E0ADE6B0E08D939C9380E082
:1010900090E0ABE6B0E08D939C9384EF91E078D242
:1010A0008EB5887F8EBD882783BFE5E0F0E0A5E799
:1010B000B0E092E07BE7AAD229C0043009F026C054
:1010C00080918C00816080938C0082E090E0AFE69C
:1010D000B0E08D939C938EE090E0ADE6B0E08D9310
:1010E0009C9380E090E0ABE6B0E08D939C9384EF1E
:1010F00091E04ED28EB5887F8EBD882783BFEAE00F
:10110000F0E0A9E7B0E092E07BE780D280918C002C
:101110008D7F80938C0080918C008E7F80938C00DB
:10112000089580918C00806280938C00A5E7B0E0E8
:101130004D915C91A3E7B0E00D911C910417150748
:1011400009F059C080918C00826080938C008FE000
:1011500090E0A5E6B0E08D939C9380E190E0A7E657
:10116000B0E08D939C9380E190E0A9E6B0E08D9390
:101170009C9384EF91E00CD28BE090E0A5E6B0E088
:101180008D939C938BE090E0A7E6B0E08D939C93C9
:101190008BE090E0A9E6B0E08D939C9384EF91E022
:1011A000F7D18FE090E0A5E6B0E08D939C9380E1CD
:1011B00090E0A7E6B0E08D939C9380E190E0A9E6F3
:1011C000B0E08D939C9384EF91E0E2D18BE090E0CE
:1011D000A5E6B0E08D939C938BE090E0A7E6B0E0AD
:1011E0008D939C938BE090E0A9E6B0E08D939C9367
:1011F00084EF91E0CDD1ABE7B0E04D915C91A9E7F0
:10120000B0E00D911C910417150709F059C08091A9
:101210008C00816080938C008FE090E0ABE6B0E0C2
:101220008D939C9380E190E0ADE6B0E08D939C932C
:1012300080E190E0AFE6B0E08D939C9384EF91E085
:10124000A7D18BE090E0ABE6B0E08D939C938BE070
:1012500090E0ADE6B0E08D939C938BE090E0AFE63C
:10126000B0E08D939C9384EF91E092D18FE090E079
:10127000ABE6B0E08D939C9380E190E0ADE6B0E00A
:101280008D939C9380E190E0AFE6B0E08D939C93CA
:1012900084EF91E07DD18BE090E0ABE6B0E08D9300
:1012A0009C938BE090E0ADE6B0E08D939C938BE057
:1012B00090E0AFE6B0E08D939C9384EF91E068D12D
:1012C00000918B00003009F001C027C0013009F007
:1012D00007C0E0E0F0E0A3E7B0E092E0A8D11DC0D5
:1012E000023009F007C0E5E0F0E0A5E7B0E092E0E9
:1012F0009ED113C0033009F007C0EAE0F0E0A9E78F
:10130000B0E092E094D109C0043009F006C0EEE0EC
:10131000F0E0ABE7B0E092E08AD180918B008150A1
:1013200080938B0080E090E0ADE8B0E08D939C93DB
:1013300080918C008F7D80938C000895789489B77C
:10134000816089BF82E083BF80E090E0ADE8B0E0DB
:101350008D939C9300918B00013009F00DC0A3E7A1
:10136000B0E00D911C91043650E0150708F003C061
:10137000A3E7B0E0B9D02FC0023009F00DC0A5E757
:10138000B0E00D911C91043650E0150708F003C041
:10139000A5E7B0E0A9D01FC0033009F00DC0A9E750
:1013A000B0E00D911C91073E53E0150708F003C013
:1013B000A9E7B0E099D00FC0043009F00CC0ABE74A
:1013C000B0E00D911C91073E53E0150708F003C0F3
:1013D000ABE7B0E089D08FE090E0DAD00895789460
:1013E00089B7816089BF82E083BF80E090E0ADE88B
:1013F000B0E08D939C9300918B00013009F00FC0F9
:10140000A3E7B0E00D911C91003050E0150710F0FB
:1014100009F001C003C0A3E7B0E06DD035C00230D1
:1014200009F00FC0A5E7B0E00D911C91003050E02D
:10143000150710F009F001C003C0A5E7B0E05BD0CC
:1014400023C0033009F00FC0A3E7B0E00D911C9159
:10145000003050E0150710F009F001C003C0A9E703
:10146000B0E049D011C0043009F00EC0ABE7B0E0E5
:101470000D911C91003050E0150710F009F001C0EB
:1014800003C0ABE7B0E037D08FE090E081D00895A3
:1014900080918C00806480938C0091E0AFE8B0E094
:1014A0008FD08EB5887F8EBD882783BFE0E1F0E0C6
:1014B000AFE8B0E091E07BE7A9D0089580918C007F
:1014C000806480938C0091E0A0E9B0E079D08EB583
:1014D000887F8EBD882783BFE1E1F0E0A0E9B0E01E
:1014E00091E07BE793D00895ED91FC91EF5FFF4F82
:1014F000FC93EE930895ED91FC91E150F040FC9344
:10150000EE93089500FC10D0089503D01ED001F88A
:10151000F9CF0024E89457FF02C009D0689400F87E
:101520000BD010F80124089502D009D008955095E9
:1015300040954F5F5F4F0895E89417FF0895009519
:1015400010950F5F1F4F68940895352F242FE8944E
:10155000452B11F468940895512F402F002711272F
:1015600080E1440F551F001F111F021B130B416028
:1015700018F4020F131F4E7F8A9599F7089531973B
:10158000F1F70895689462F80895E89462F8089570
:10159000EF93FF93EE27E82BE92B31F0E0EDF7E036
:1015A0003197F1F70197D1F7FF91EF910895369AAE
:1015B0003699FECF369A3699FECF84B195B108950B
:1015C000903039F08C91880F08F481609A95D9F7A2
:1015D0008C930895C89531960020089591E005C038
:1015E00092E003C094E001C098E0F4DF0D929A9578
:1015F000E1F70895E80FF91FF1CFE199FECFEEBBB7
:10160000FFBB3196089591E001C092E07B3751F421
:101610007FB7F894F2DF8D918DBBE29AE19A9A95AB
:10162000C9F77FBF7727089591E001C092E0E5DF19
:0C163000E09A8DB38D939A95D1F7089540
:00000001FF
